:100000000C9461000C947E000C947E000C947E0095
:100010000C947E000C947E000C947E000C947E0068
:100020000C947E000C947E000C947E000C947E0058
:100030000C947E000C947E000C947E000C947E0048
:100040000C949A000C947E000C947E000C947E001C
:100050000C947E000C947E000C947E000C947E0028
:100060000C947E000C947E00000000002400270009
:100070002A0000000000250028002B0000000000DE
:1000800023002600290004040404040404040202DA
:100090000202020203030303030301020408102007
:1000A0004080010204081020010204081020000012
:1000B0000007000201000003040600000000000029
:1000C000000011241FBECFEFD8E0DEBFCDBF11E08E
:1000D000A0E0B1E0E4E5F4E002C005900D92A030AC
:1000E000B107D9F711E0A0E0B1E001C01D92A9303D
:1000F000B107E1F70E9418020C9428020C9400004A
:1001000086E061E00E94C4016AEF70E080E090E068
:100110000E941D0186E060E00E94C4016AEF70E069
:1001200080E090E00E941D01089586E061E00E9459
:10013000850108951F920F920FB60F9211242F93ED
:100140003F938F939F93AF93BF93809104019091BE
:100150000501A0910601B0910701309108010196B7
:10016000A11DB11D232F2D5F2D3720F02D57019696
:10017000A11DB11D209308018093040190930501F6
:10018000A0930601B09307018091000190910101B5
:10019000A0910201B09103010196A11DB11D8093B0
:1001A000000190930101A0930201B0930301BF915C
:1001B000AF919F918F913F912F910F900FBE0F9014
:1001C0001F901895789484B5826084BD84B5816051
:1001D00084BD85B5826085BD85B5816085BDEEE64F
:1001E000F0E0808181608083E1E8F0E0108280812E
:1001F00082608083808181608083E0E8F0E080819C
:1002000081608083E1EBF0E0808184608083E0EBBB
:10021000F0E0808181608083EAE7F0E080818460A3
:1002200080838081826080838081816080838081FF
:10023000806880831092C1000895EF92FF920F931F
:100240001F93CF93DF937B018C013FB7F89480918C
:10025000000190910101A0910201B091030126B526
:10026000A89B05C02F3F19F00196A11DB11D3FBFEE
:10027000BA2FA92F982F8827820F911DA11DB11D7C
:1002800052E0880F991FAA1FBB1F5A95D1F7EC01A6
:1002900030C00E9427023FB7F894809100019091EE
:1002A0000101A0910201B091030126B5A89B05C0F0
:1002B0002F3F19F00196A11DB11D3FBFBA2FA92FE5
:1002C000982F8827820F911DA11DB11D32E0880F44
:1002D000991FAA1FBB1F3A95D1F78C1B9D0B885EF7
:1002E0009340B8F20894E108F10801091109C851D6
:1002F000DC4FE114F1040105110559F6DF91CF91AE
:100300001F910F91FF90EF900895CF93DF93482FA7
:1003100050E0CA0186569F4FFC0134914A575F4F07
:10032000FA018491882369F190E0880F991FFC01FC
:10033000E859FF4FA591B491FC01EE58FF4FC591CC
:10034000D491662351F42FB7F8948C91932F909504
:1003500089238C93888189230BC0623061F42FB785
:10036000F8948C91932F909589238C938881832B7B
:1003700088832FBF06C09FB7F8948C91832B8C93F2
:100380009FBFDF91CF910895482F50E0CA01825559
:100390009F4FFC012491CA0186569F4FFC01949106
:1003A0004A575F4FFA013491332309F440C02223A6
:1003B00051F1233071F0243028F42130A1F02230A3
:1003C00011F514C02630B1F02730C1F02430D9F433
:1003D00004C0809180008F7703C0809180008F7D62
:1003E0008093800010C084B58F7702C084B58F7D64
:1003F00084BD09C08091B0008F7703C08091B000A8
:100400008F7D8093B000E32FF0E0EE0FFF1FEE58DA
:10041000FF4FA591B4912FB7F894662321F48C91E6
:100420009095892302C08C91892B8C932FBF0895BE
:10043000CF93DF930E94E2000E949500C0E0D0E0DD
:100440000E9480002097E1F30E940000F9CF0895F8
:04045000F894FFCF4E
:00000001FF
